:100000000C94C6010C9419020C9419020C94190258
:100010000C9419020C9419020C9419020C941902F4
:100020000C9419020C9419020C94391C0C940B1D9D
:100030000C942A210C9419020C9419020C941902A4
:100040000C9419020C9419020C9419020C941902C4
:100050000C9419020C941C080C9419020C941902AB
:100060000C9419020C9419020C9419020C941902A4
:100070000C9419020C9419020C9419020C94190294
:100080000C9419020C9419020C9419020C94190284
:100090000C9419020C9419020C9419020C94190274
:1000A0000C9419020C9419020C941902871AAE1AB6
:1000B000A61BAE1AA61BFA1A1D1BA61B741B831BBC
:1000C0007573625F73746174653A20253032580A23
:1000D000000D0A2F2F2050617273652064617461D6
:1000E00020686572653A20687474703A2F2F656CC9
:1000F000656363656C657261746F722E636F6D2FDB
:100100007573626465736372657170617273657231
:100110002F0D0A000D0A2F2F204465766963652094
:1001200044657363726970746F723A0D0A000D0A48
:100130002F2F206953657269616C4E756D6265720F
:100140003A20000D0A2F2F206950726F6475637476
:100150003A20000D0A2F2F20694D616E756661638C
:1001600074757265723A20000D0A2F2F2053747235
:10017000696E67303A0D0A002F2F206C6F7773700D
:100180006565643A253032580D0A000D0A2F2F207C
:10019000416464726573733A253032580D0A000D5C
:1001A0000A2F2F2069436F6E6669677572617469E3
:1001B0006F6E3A2000427566666572206973206E24
:1001C0006F7420656E6F756768210D0A000D0A2F28
:1001D0002F20436F6E66696725643A000D0A2F2F42
:1001E000205265706F727425643A206C656E3A25F2
:1001F0003034580D0A000D0A2F2F2069496E74659E
:1002000072666163653A20000D0A000D0A0053749E
:1002100072696E6725643A20000D0A002530325855
:1002200020002F2F20000D0A0020000D0A455252F9
:100230004F523A253032580D0A0025733A25303492
:10024000580D0A0025733A253032580D0A00253022
:1002500032580000000D0A0020000A4B6579626FD9
:100260006172642073746172742E0A000A555342DD
:1002700020636F6E666967757265642E0A000A0AEC
:10028000544D4B3A66623665653130662B2F4C55BE
:1002900046410A0A002C0355005300420020004446
:1002A0000065007300630072006900700074006FE5
:1002B0000072002000440075006D0070006500723F
:1002C000000000080354004D004B00000004030927
:1002D0000409024200020100A032090400000103E7
:1002E00001010009211101000122400007058103DD
:1002F00008000A090401000203000000092111019D
:1003000000012222000705820320000107050203E5
:100310002000011201100100000008EDFE5B001436
:1003200008010200010631FF0974A10109751500D9
:1003300026FF009520750881020976150026FF002A
:10034000952075089102C005010906A1010507194C
:10035000E029E715002501950875018102950175D1
:100360000881010508190129059505750191029576
:1003700001750391010507190029FF150026FF00EB
:10038000950675088100C0005F07870711241FBE0E
:10039000CFEFDAE0DEBFCDBF04B603FE28C0809108
:1003A000C7059091C805A091C905B091CA058730CD
:1003B000904BA740B04BD9F41092C7051092C805D6
:1003C0001092C9051092CA0514BE0FB6F894A895EC
:1003D00080916000886180936000109260000FBE81
:1003E0001092010810920008E0E0F8E3099511E08E
:1003F000A0E0B1E0E8E5F7E402C005900D92A63A6E
:10040000B107D9F725E0A6EAB1E001C01D92A73CEB
:10041000B207E1F711E0C6ECD1E004C02197FE017C
:100420000E94A423C43CD107C9F70E94A2170C94D0
:10043000AA230C940000FF93EF93E091A601F091A2
:10044000A701309709F00995EF91FF910895FC01FC
:100450008591803011F0EFDFFBCF0895FF27E0E2B8
:1004600030E247FF0CC0419597FF09C0EDE260956F
:10047000709580959095611D711D811D911D27FFBF
:1004800002C0219530E350E2AA27660F771F881F2C
:10049000991FAA1FA41710F0A41B63955A95A9F7DA
:1004A000AA3008F0A95FA05DAF93F39561157105BF
:1004B0008105910541F7ED3211F4EF93F395F217B1
:1004C00018F43F93F395FBCF8F91B5DFFA95E1F7E1
:1004D0000895E991F9918591803021F0853219F0E4
:1004E000AADFF9CF089520E0E89455915532C1F381
:1004F000503311F4689455915A3348F4505390F3A3
:10050000220F022E220F220F200D250FF4CF0EF402
:10051000219589919991533619F3533729F1533520
:1005200059F1BC0188279927E8945C3621F4899118
:10053000999168945591543639F446EF7EF077FFDF
:100540000DC08FEF9FEF0AC055374AE039F058359C
:1005500040E121F0523642E009F00895FF93EF9315
:100560007DDFEF91FF91B7CFFF93EF93FC01819176
:100570008030B9F360DFFBCFFF93EF9368DFF1CFFB
:10058000DF93CF93CDB7DEB72596A3DFCF91DF9171
:1005900008951F928F938EE492E09F938F930E9411
:1005A000C0020F900F900F900F900895CF92DF929E
:1005B000EF92FF920F931F93CF93DF936B0179011B
:1005C0008A01C0E0D0E0CC15DD05D1F0F7018081D3
:1005D00091818C0F9D1F9C012F703327232B19F0C5
:1005E00088E592E004C0892B21F085E592E00E9425
:1005F0002702F80181918F010E94C9022196E3CF61
:10060000DF91CF911F910F91FF90EF90DF90CF90EE
:1006100008951F926F939F938F9384E492E09F932A
:100620008F930E94C0020F900F900F900F900F9029
:100630000F9008957F936F939F938F938AE392E037
:100640009F938F930E94C0020F900F900F900F9076
:100650000F900F9008951F928F938BE292E09F93DB
:100660008F930E94C0020F900F900F900F900895EB
:10067000BF92CF92DF92EF92FF920F931F93CF938F
:10068000DF936C01B42E8B01C0E0D0E08CE1E82E4A
:1006900082E0F82ECC15DD051CF5CE018F70992770
:1006A000892B19F089E292E00AC0209721F086E2B6
:1006B00092E00E942702BB2021F082E292E00E9499
:1006C0002702F80181918F011F928F93FF92EF9281
:1006D0000E94C00221960F900F900F900F90DACFDA
:1006E00089E192E0DF91CF911F910F91FF90EF9000
:1006F000DF90CF90BF900C9427026F927F928F92E1
:100700009F92AF92BF92CF92DF92EF92FF920F93A0
:100710001F93CF93DF93CDB7DEB7DA950FB6F8947A
:10072000DEBF0FBECDBF662309F45CC03A01162FB1
:100730004C01CE0101966C017A01062F21E030E0D8
:1007400040E0F401628184EC93E00E948B0E811101
:1007500011C0A980B12CCE0101966C017301012F4B
:10076000950140E0F401628184EC93E00E948B0EDD
:10077000882319F00E942B0335C01F921F938EE02F
:1007800092E09F938F930E94C0020F900F900F9062
:100790000F9012E0812F90E09C012F5F3F4F2A15B0
:1007A0003B05A4F4E1E0F0E0EC0FFD1FE20FF31FC6
:1007B0002081211109C0E1E0F0E0EC0FFD1FE80FFE
:1007C000F91F80810E941B021E5FE4CF8BE092E044
:1007D0000E942702898141E0BE016F5F7F4F90E058
:1007E0000E943803D3950FB6F894DEBF0FBECDBF7D
:1007F000DF91CF911F910F91FF90EF90DF90CF90FD
:10080000BF90AF909F908F907F906F9008958F9240
:100810009F92AF92BF92CF92EF920F931F93CF937D
:10082000DF93CDB7DEB7C054D1090FB6F894DEBF61
:100830000FBECDBF2CEA31E03F932F939E012F5F77
:100840003F4F3F932F931F9220E42F934A015B0168
:1008500022E2C22EE12C06E021E840E0FC016281A8
:1008600084EC93E00E945D0D182F88E092E00E94D6
:1008700027020F900F900F900F900F900F90112361
:1008800019F0812F0E942B03812FC05CDF4F0FB620
:10089000F894DEBF0FBECDBFDF91CF911F910F91B6
:1008A000EF90CF90BF90AF909F908F9008958F92D0
:1008B0009F92AF92BF92CF92DF92EF92FF921F93DF
:1008C000CF93DF936C01EA0110E0CB018D549E4F72
:1008D0007C018CEDA82E81E0B82ECE15DF0508F046
:1008E00056C06981613178F46F3008F04CC06430D3
:1008F000B1F020F4613008F442C045C0653009F41D
:1009000042C086EF08C0663228F46432E0F56132F6
:10091000B9F035C080ED860F823088F534C01A8179
:100920008885882381F186EF91E00E94270240911B
:10093000B1015091B2016885C6010E947D0323C0B8
:1009400088858F938F818F93812E912C1F921F9377
:10095000BF92AF920E94C0026E810F900F900F90D5
:100960000F900F900F90623239F44F815885B40187
:10097000C6010E94070407C085E191E002C08FE232
:1009800091E00E9409038881C80FD11DA6CFDF9195
:10099000CF911F91FF90EF90DF90CF90BF90AF90DD
:1009A0009F908F9008956F927F928F929F92AF92B7
:1009B000BF92CF92DF92EF92FF920F931F93CF934C
:1009C000DF936C01862E912CC0E0D0E03DEC632ECD
:1009D00031E0732E1C2F8C169D0609F46FC0DF9337
:1009E000CF937F926F920E94C00223EBE22E21E010
:1009F000F22E0C2F29E030E040E0F601628184EC19
:100A000093E00E94640E0F900F900F900F90811151
:100A100056C06091B5017091B60185E491E00E94E5
:100A20001A03A090B501B090B601F1E0AF16F2E064
:100A3000BF0618F0A12C92E0B92E83EBE82E81E0DE
:100A4000F82E012F950140E0F601628184EC93E0DD
:100A50000E94640E811133C040E0B701C5010E94BD
:100A600038038091B5019091B6018130924020F019
:100A700085EB91E00E9427028091B901882369F0FB
:100A80008FE991E00E9427024091B1015091B2019B
:100A90006091B901C6010E947D032091B80140E038
:100AA000F601628184EC93E00E94211043EB51E057
:100AB000B501C6010E94570421968CCF80E0DF91DA
:100AC000CF911F910F91FF90EF90DF90CF90BF904B
:100AD000AF909F908F907F906F900895AF92BF924C
:100AE000CF92DF92EF92FF920F931F93CF93DF93FA
:100AF00000D000D0CDB7DEB75C01DC0112968C913E
:100B00001F928F938BE891E09F938F930E94C00276
:100B1000F50184811F928F9388E791E09F938F93D3
:100B20000E94C00203EB11E022E130E040E0D50179
:100B300012966C9184EC93E00E943D0E0FB6F894EF
:100B4000DEBF0FBECDBF81110E942B036091BB01A0
:100B50007091BC018AE491E00E941A036091BD018A
:100B60007091BE0186E591E00E941A031092AE01D9
:100B70008091BA018093AF018091B00183708C6342
:100B80008093B001E091C403F091C5030190F0811E
:100B9000E02DD50112966C9184EC93E009952EEA34
:100BA00031E0FC01318320838091C101811108C0B3
:100BB0008091C201811104C08091C301882339F161
:100BC0009E012F5F3F4F6901E12CF12C00E024E0F2
:100BD00030E040E0D50112966C9184EC93E00E94E5
:100BE0008B0E811114C06B817C817093B201609374
:100BF000B10183E691E00E941A0388E691E00E9429
:100C00002702898141E0B60190E00E94380380917B
:100C1000C101882369F083E591E00E942702409199
:100C2000B1015091B2016091C101C5010E947D03E3
:100C30008091C201882369F083E491E00E94270239
:100C40004091B1015091B2016091C201C5010E9471
:100C50007D038091C301882369F08EE291E00E94B8
:100C600027024091B1015091B2016091C301C501C9
:100C70000E947D0384E191E00E94270240E063EB43
:100C800071E082E190E00E9438036091C401C501E7
:100C90000E94D30481110E942B03E091C403F091C0
:100CA000C5030480F581E02DD50112966C9184EC8A
:100CB00093E0099581ED90E00E9427020F900F903C
:100CC0000F900F90DF91CF911F910F91FF90EF90B8
:100CD000DF90CF90BF90AF90089508950E94F507E0
:100CE0009093AB018093AA01089581E00895CF937A
:100CF000DF9384EC93E00E947F1084EC93E00E94E9
:100D00004D099091A8018917C9F084EC93E00E94E5
:100D10004D098093A8011F928F9380EC90E09F93E0
:100D20008F930E94C0020F900F900F900F908091B0
:100D30000001811103C081E0809300018091AA012C
:100D40009091AB010E940D08883B9B40C8F084EC59
:100D500093E00E944D09803999F480910001882325
:100D600079F0CFECD3E08A81882319F0CE010E947C
:100D70006E05259684E0CA31D807A9F710920001C4
:100D8000DF91CF9108952E9A08952E988EBD0DB4BF
:100D900007FEFDCF1EBC0DB407FEFDCF0E94C306AB
:100DA0008EB508952E9882608EBD0DB407FEFDCFDE
:100DB0006EBD0DB407FEFDCF0C94C30688EF0E94F4
:100DC000C506807C8034A1F018F4882301F10895D1
:100DD000803819F0803CB9F0089588ED0E94C5066E
:100DE00081FD0BC069EC88ED0E94D20682E00CC048
:100DF00088ED0E94C50681FDF5CF6BEC88ED0E9461
:100E0000D20683E001C081E08093A901089561EDDD
:100E100088ED0E94D2061092A90108950F931F93A6
:100E2000CF93DF938C01269A0E94C306219A229ABF
:100E30002398209A80E58CBD81E08DBD259868E1DE
:100E400088E80E94D20660E288E70E94D20660E04D
:100E500088E70E94D206C0E0D0E088E60E94C5067E
:100E6000219680FD06C0CF3F8FEFD807B1F78FEFF7
:100E70001DC061EC88ED0E94D20660E680ED0E9404
:100E8000D20664E088EE0E94D20688EE0E94C50673
:100E900082FFFBCFC8010E94DE0660E288EC0E9460
:100EA000D20661E080E80E94D20680E0DF91CF9117
:100EB0001F910F91089584EC93E00C940E0784EC3D
:100EC00093E00E941D0964EC73E083EB93E00E94C1
:100ED000DC1381E791E09093AD018093AC0108951C
:100EE00080E090E008958FEF9FEF089581E090E01B
:100EF00008950895862F0E94961581E090E0089548
:100F0000FB0180810E94961581E090E00895EBE35B
:100F1000F4E01382128288EE93E0A0E0B0E08483D4
:100F20009583A683B78387E791E0918380838FEFD2
:100F30009FEF9587848708950C9401088F929F9264
:100F4000AF92BF92CF92DF92EF92FF920E948022E7
:100F50004B015C0120E030E04AE755E40E94372372
:100F60006B017C0120E030E040E85FE30E944C220E
:100F700087FD24C020E03FEF4FE757E4C701B601EB
:100F80000E9432231816ACF420E030E040E251E435
:100F9000C501B4010E9437230E94512220E931E0AB
:100FA0006115710581F0C9010197F1F7615071096F
:100FB000F7CFC701B6010E94512202C061E070E084
:100FC000CB010197F1F7FF90EF90DF90CF90BF90AA
:100FD000AF909F908F90089582E084BD93E095BD7F
:100FE0009AEF97BD80936E0008952FB7F894809183
:100FF0008B0490918C04A0918D04B0918E042FBF2E
:1010000008952FB7F89460918B0470918C048091AF
:101010008D0490918E042FBF08959C014FB7F894D2
:1010200080918B0490918C04A0918D04B0918E04DA
:101030004FBF821B930B089578941F920F920FB6A7
:101040000F9211248F939F93AF93BF9380918B0442
:1010500090918C04A0918D04B0918E040196A11DF5
:10106000B11D80938B0490938C04A0938D04B09356
:101070008E04BF91AF919F918F910F900FBE0F90F3
:101080001F901895CF93DF93FC01862F8078A9F4E9
:10109000283008F04DC0442321F09581973009F4A1
:1010A00047C0EF01A1E0B0E09D85992341F0119682
:1010B0002596A031B105C1F73BC080E039C0611170
:1010C0001CC085E08A9FE0018B9FD00D1124CE0FBC
:1010D000DF1F442331F081E4888785818F5F85831A
:1010E00002C081E0888725E02A9FC0012B9F900DD8
:1010F0001124E80FF91F80851BC06770660F660F0B
:10110000660F442341F0606485818F5F858387701B
:10111000687F682B03C02770687B622B25E02A9FBD
:10112000C0012B9F900D1124E80FF91F6087862FB7
:10113000DF91CF910895611102C006960895FC01D8
:1011400021E03585631739F02F5F35962031C9F7D7
:1011500080E090E00895069635E0239F800D911D74
:1011600011240895DF92EF92FF920F931F93CF9374
:10117000DF93EC01E62EF12C85E0689FB00111248D
:10118000FE01E60FF71F8085182F177086FF17C026
:1011900001E085E0D82EFE01D09EE00DF11D112466
:1011A000808586958695869587701817F9F00F5F6C
:1011B000003189F78D81811302C011501D8385E0B4
:1011C0008E9DF0018F9DF00D1124EC0FFD1F1086F8
:1011D00081E0818712862296D783C683DF91CF91E3
:1011E0001F910F91FF90EF90DF900895602FCE0137
:1011F0000E94B208D0CFFC01613499F49C01255BB8
:101200003F4F61E0AC014E5F5F4F158666871786E2
:10121000548743873596E217F307B9F7FC01158227
:10122000089521E03585631729F02F5F3596203129
:10123000C9F70895622F0C94B208FC0189E891E087
:10124000918380831582108681E081871286CF0189
:10125000029697838683128228E023832CE32483DB
:10126000DF019F01255B3F4F41E01D961C921D97BA
:101270001E964C931E971F961C921F971C969C932C
:101280008E931B971596A217B30779F7EA58FF4F6D
:10129000108281E1809393040895809193040895CE
:1012A000CF93C42F0E949B08009789F0DC01ED9139
:1012B000FC911197309759F013969C9180E0891713
:1012C00031F020812C1731F033968F5FF8CF80E01A
:1012D00090E001C0CF01CF9108950F931F93CF935A
:1012E000DF932115310571F0E901042F162F0E94BB
:1012F0009B08FC01892B41F01283D183C0830383B7
:1013000080E003C088ED01C086EDDF91CF911F9191
:101310000F910895CF92DF92FF920F931F93CF9377
:10132000DF93662381F1F62E8C016C0186E5C80EF1
:10133000D11CC0E0D0E0D6018D919D916D01009748
:10134000F1F0DC01ED91FC910084F185E02D09952F
:10135000F81215C0AB96CC0FDD1FC00FD11F8881CE
:101360009981DC01ED91FC910480F581E02DDF9104
:10137000CF911F910F91FF90DF90CF90099421960C
:10138000C031D105C1F680E0DF91CF911F910F915F
:10139000FF90DF90CF9008952E980895CF93C82F97
:1013A0000E94CC09CEBD0DB407FEFDCF1EBC0DB40E
:1013B00007FEFDCF0E94C3068EB5CF910895CF934F
:1013C000DF93C82FD62F0E94CC09C260CEBD0DB4CA
:1013D00007FEFDCFDEBD0DB407FEFDCFDF91CF913F
:1013E0000C94C3068F929F92AF92BF92CF92DF92DE
:1013F000EF92FF920F931F93CF93DF93EC01D62EC2
:10140000C42E59010E949B087C01009709F445C035
:10141000FC0180819181892B09F441C04C2D6D2DF7
:10142000CE010E945009F501918380830097C9F194
:10143000FC0182818695869590E08031910514F0BB
:101440008FE090E041E050E060E070E04A015B0135
:1014500004C0880C991CAA1CBB1C8A95D2F7D50124
:10146000C4010197F801918380836D2D80EE0E9465
:10147000DF0988ED0E94CE09F7019481992331F0AC
:10148000CA58DF4F68816260682B02C0682F697F8D
:1014900088ED0E94DF0980E005C086ED03C087ED7E
:1014A00001C08BEDDF91CF911F910F91FF90EF90D5
:1014B000DF90CF90BF90AF909F908F9008958F92C4
:1014C0009F92AF92BF92CF92DF92EF92FF920F93D3
:1014D0001F93CF93DF93862E942E59010E949C0771
:1014E0006B017C0128E8C20E23E1D21EE11CF11C35
:1014F00000E010E0D0E0C0E098280E949C07DC01EA
:10150000CB018C199D09AE09BF09B7FF2DC0692D0C
:1015100080EF0E94DF090E949C07DC01CB018C193F
:101520009D09AE09BF09B7FF09C088EC0E94CE092A
:1015300087FFF1CF60E888EC0E94DF0988EF0E9406
:10154000CE09C82FCF70C43019F0CE3051F00CC086
:101550000F5F1F4FA114B10481F20A151B0569F634
:1015600003C0DF5FD33049F68C2FDF91CF911F91FD
:101570000F91FF90EF90DF90CF90BF90AF909F9032
:101580008F9008959F92AF92BF92CF92DF92EF9289
:10159000FF920F931F93CF93DF937C01D42F122FD1
:1015A000902E00E06C01C60ED11CC60ED11C86E543
:1015B000C80ED11CA42EB12CABE2AA0EB11CAA0CF1
:1015C000BB1CAE0CBF1CF60180819181DC01ED914A
:1015D000FC910280F381E02D292D412F6D2F09957B
:1015E000803EC9F4D1110BC061E088EE0E94DF0992
:1015F00066E670E080E090E00E949E0714C0F5016E
:1016000080819181DC01ED91FC910284F385E02DD4
:10161000612F099508C08D3021F4033008F03FC0D8
:1016200014C081113FC0F60180819181DC01ED91F0
:10163000FC910190F081E02D292D412F6D2F09950E
:10164000C82F8D3051F4033050F464E670E080E030
:1016500090E00E949E070F5FB6CF882311F1D11151
:101660000BC061E088EE0E94DF0966E670E080E072
:1016700090E00E949E0711C0ED2FF0E0BB96EE0FA8
:10168000FF1FEE0DFF1D80819181DC01ED91FC912A
:101690000284F385E02D612F09958C2F03C08DE026
:1016A00001C080E0DF91CF911F910F91FF90EF90EB
:1016B000DF90CF90BF90AF909F9008950F931F93AE
:1016C000CF93DF93182F062FEA010E94CC091260F6
:1016D0001EBDFE01802F882339F00DB407FEFDCF1B
:1016E00091919EBD8150F7CFC00FD11D0DB407FE63
:1016F000FDCF0E94C306CE01DF91CF911F910F91C4
:1017000008952F923F924F925F926F927F928F92A5
:101710009F92AF92BF92CF92DF92EF92FF920F9380
:101720001F93CF93DF9300D000D01F92CDB7DEB7C9
:101730007D836C834A016901FB01F1808FEF8F0D7E
:10174000803408F067C00E949C072B013C01F8E838
:101750004F0EF3E15F1E611C711CEC81FD818281E3
:1017600080FD02C060E401C060E888EE0E94DF09ED
:10177000312C8F2D90E09A838983C114D104B1F16B
:10178000E980FA80CE14DF0408F47601EB82A80128
:101790006E2D80E10E945E0B6E2D88E30E94DF09B2
:1017A000EC81FD816081606280EF0E94DF0988EC3E
:1017B0000E94CE0987FFFBCF60E888EC0E94DF091A
:1017C00088EF0E94CE098F70382EA12CB12C212CCD
:1017D000332009F472C00E949C07DC01CB018419FC
:1017E0009509A609B709B7FF68C016C0332021F0D4
:1017F00060E088E30E94DF0988EF0E94CE0985FB44
:10180000882780F9EC81FD81928180FB90F9928399
:10181000832D58C08AED56C0F6E03F1239C088EFDC
:101820000E94CE0985FB882780F991E08927EC8109
:10183000FD81928180FB90F9928390FD02C060E46B
:1018400001C060E888EE0E94DF0960E088E30E9442
:10185000DF09F801608180E10E94DF096B8188E384
:101860000E94DF09EC81FD816081606280EF0E944F
:10187000DF0988EC0E94CE0987FFFBCF60E888EC87
:101880000E94DF0988EF0E94CE098F70382EA0CF0A
:101890002EE0321205C0239423E02212D6CFA8CF27
:1018A00084E03812A5CFFFEFAF1ABF0A811491046C
:1018B00061F2A814B90449F69BCFCE18DF080E0DCB
:1018C0001F1D5BCF0F900F900F900F900F90DF9127
:1018D000CF911F910F91FF90EF90DF90CF90BF902D
:1018E000AF909F908F907F906F905F904F903F90C0
:1018F0002F9008952F923F924F925F926F927F9216
:101900008F929F92AF92BF92CF92DF92EF92FF920F
:101910000F931F93CF93DF93CDB7DEB72A970FB600
:10192000F894DEBF0FBECDBF1C016B015B834A8301
:101930005901D9016D907C901197FB01F181F983D8
:101940001D921C92DB0112968C9181FD02C060E118
:1019500001C060E288EE0E94DF098E2D90E0A0E0D9
:10196000B0E08C839D83AE83BF8368862A813B81F0
:10197000D6014C9160E0C1010E945F0AF82EB6E0EA
:101980008B1318C088EF0E94CE0982958170E1E028
:101990008E27D60112969C91129780FB91F9129690
:1019A0009C9391FD02C060E101C060E288EE0E945C
:1019B000DF09DCCF811167C088EC0E94CE0982FF6D
:1019C00060C080E30E94CE09582E90E06816790628
:1019D00008F45884F501808191819301281B390B0B
:1019E0003A87298737FF02C01A861986852C912CE1
:1019F00089859A858816990614F49A868986498479
:101A00000E94CC0998E09EBD0DB407FEFDCFF80101
:101A1000442041F01EBC4A940DB407FEFDCF8EB5A4
:101A20008193F6CFA985BA850A0F1B1F0E94C306B2
:101A300064E088EC0E94DF09F50180819181880EC5
:101A4000991E91828082F9815F1618F0861497049E
:101A500070F088EF0E94CE0982958170D6011296AF
:101A60009C91129780FB91F912969C930CC0EE20EA
:101A700009F47CCF6C817D818E819F810E949E07BD
:101A800075CF80EFF82E8F2D2A960FB6F894DEBF13
:101A90000FBECDBFDF91CF911F910F91FF90EF90BF
:101AA000DF90CF90BF90AF909F908F907F906F907E
:101AB0005F904F903F902F9008952F923F924F92BA
:101AC0005F926F927F928F929F92AF92BF92CF92CE
:101AD000DF92EF92FF920F931F93CF93DF93CDB7D7
:101AE000DEB761970FB6F894DEBF0FBECDBF3C01E5
:101AF000F42E322E202EC98A4EA05FA0C8A4D9A4ED
:101B0000188A1F861E861D868E01035F1F4F9E0149
:101B1000215F3F4F0E94F209811196C039822A82CB
:101B2000EB8289898C83BE82AD8298868F82AE01DA
:101B30004F5F5F4F68E080E20E945E0B2D853E851F
:101B40004F2D60E1C3010E945F0AE82E811178C029
:101B5000932D9078392EC114D10409F462C0EF8519
:101B6000F8898281992309F44DC0826082835401EF
:101B700022242394A114B10409F458C05C864B8636
:101B80004D855E856F857889E12C86019E01255FF4
:101B90003F4FC3010E947A0CE82EA6E08A130FC0C3
:101BA0000F85188988EF0E94CE0985FB882780F968
:101BB0008225F801928180FB91F99283DBCF81111C
:101BC0003FC08AA59BA50097A1F0DC01ED91FC9197
:101BD00011970190F081E02DC4018A199B099A8721
:101BE00089876B857C859E01275F3F4FA601CD01CC
:101BF00009958B859C85A81AB90A8415950508F066
:101C0000B9CF0FC0816082834D855E8586019201C8
:101C1000BF01C3010E94810B811116C02D853E8535
:101C200011C02D853E85311005C00CC0E11008C0E3
:101C30002D853E8560EA4F2DC3010E945F0A04C0D6
:101C40008E2D02C060E8F7CF61960FB6F894DEBF24
:101C50000FBECDBFDF91CF911F910F91FF90EF90FD
:101C6000DF90CF90BF90AF909F908F907F906F90BC
:101C70005F904F903F902F9008958F929F92AF92D8
:101C8000BF92CF92EF920F931F931F921F921F93B9
:101C90000F933F932F934901A12CB12CCC24C394D3
:101CA000E12C06E020E80E945D0D0F900F900F9050
:101CB0000F900F900F901F910F91EF90CF90BF90CA
:101CC000AF909F908F9008958F929F92AF92BF9206
:101CD000CF92EF92FF920F931F921F92FF92EF927B
:101CE0003F932F934901A12CB12C22E0C22EE02E6C
:101CF00006E020E80E945D0D0F900F900F900F906E
:101D00000F900F900F91FF90EF90CF90BF90AF90FA
:101D10009F908F9008958F929F92AF92BF92CF9293
:101D2000DF92EF92FF920F931F921F92DF92CF925A
:101D30003F932F934901570123E0C22EE02E06E086
:101D400020E80E945D0D0F900F900F900F900F9064
:101D50000F900F91FF90EF90DF90CF90BF90AF90DA
:101D60009F908F9008958F929F92AF92BF92CF9243
:101D7000EF920F93CF931F921F921F921F921F9269
:101D80001F92812C912CA12CB12CC12CE22E05E0AC
:101D900020E00E945D0DC82F6CE271E080E090E0D1
:101DA0000E949E070F900F900F900F900F900F9032
:101DB0008C2FCF910F91EF90CF90BF90AF909F90CD
:101DC0008F9008950F931F93CF93DF938A3F3FEF38
:101DD000930711F486ED2DC0DC011696ED91FC9170
:101DE0001797EF2B09F1122F242FEC011A8740E0EF
:101DF0000E944208082F8823C9F0682FCE010E9454
:101E00009B08009739F3FC011483202F40E060E029
:101E1000CE010E94B30E182F882351F0602FCE01FF
:101E20000E94FB08812F05C087ED03C084ED01C02F
:101E300080E0DF91CF911F910F9108952F923F92F3
:101E40004F925F926F927F928F929F92AF92BF92CA
:101E5000CF92DF92EF92FF920F931F93CF93DF9376
:101E6000CDB7DEB766970FB6F894DEBF0FBECDBF15
:101E70001B8A38E03C8B3CE33D8B8A3F3FEF930766
:101E800009F464C0522E342E462E7C01DC011696D5
:101E9000CD90DC901797CE01439617969C938E9326
:101EA00016971A962C938E010F5F1F4F22E130E098
:101EB00040E060E0C7010E943D0EF701D782C68274
:101EC0008111A6C089849A846B847C84FD81FE8BF9
:101ED0002E80670136E5C30ED11C560110E0D501F6
:101EE0008D919C910097F1F1DC01ED91FC910084C2
:101EF000F185E02D0995811135C0F5018081918131
:101F0000DC01ED91FC910088F189E02D622D0995AD
:101F1000882341F1F50180819181DC01ED91FC91F3
:101F20000484F585E02DA301B4010995811110C049
:101F3000F50180819181DC01ED91FC910684F785AA
:101F4000E02D6E890995811103C00CC086ED60C03B
:101F5000052D232D442D612FC7010E94C20A813D0A
:101F600009F056C01F5FB2E0AB0EB11C103109F092
:101F7000B6CF10E0F601808191810097E1F1DC019C
:101F8000ED91FC910084F185E02D0995811133C01C
:101F9000F60180819181DC01ED91FC910088F1894D
:101FA000E02D622D09958823D9F0F6018081918179
:101FB000DC01ED91FC910484F585E02DA301B401D1
:101FC0000995811118C0F60180819181DC01ED91A4
:101FD000FC910684F785E02D6E89099581110BC06F
:101FE000052D232D442D612FC7010E94C20A982F71
:101FF000977F913D69F41F5FE2E0CE0ED11C103156
:1020000009F0B8CF252D432D642DC7010E94E20EA3
:1020100066960FB6F894DEBF0FBECDBFDF91CF91AD
:102020001F910F91FF90EF90DF90CF90BF90AF90F6
:102030009F908F907F906F905F904F903F902F90E8
:1020400008958F929F92AF92BF92CF92EF920F938B
:102050001F921F921F921F921F921F92812C912CF0
:10206000A12CB12CC12CE22E09E020E00E945D0DD4
:102070000F900F900F900F900F900F900F91EF9087
:10208000CF90BF90AF909F908F9008958F929F9226
:10209000AF92BF92CF92DF92EF920F931F93CF93A5
:1020A000DF9300D000D0CDB7DEB76C0159014801F5
:1020B0001C821B821A8219828E010F5F1F4F9E01A4
:1020C0002D5F3F4F0E94F209811109C049815A8159
:1020D0006B817C8184019501C6010E947A0C0F906E
:1020E0000F900F900F90DF91CF911F910F91EF9074
:1020F000DF90CF90BF90AF909F908F900895AF9258
:10210000BF92CF92DF92EF92FF920F931F93CF93E4
:102110008C011D990EC088EC0E94CE0985FF05C078
:10212000C8010E94DE0660E201C060E088EC0E9407
:10213000DF098091A901813039F040F0823079F0D7
:10214000833039F5C1E00CC083E106C0809193046F
:10215000807F8031F1F081E1809393041AC0C0E068
:1021600080919304807F8031A9F40E949C07DC0158
:10217000CB0188539F4FAF4FBF4F80938F049093F5
:102180009004A0939104B093920480E2809393040E
:1021900001C0C0E0780186E5E80EF11C6801A6E701
:1021A000CA0ED11C5701F501819191915F010097F1
:1021B00039F0DC01ED91FC910680F781E02D099565
:1021C000AC14BD0481F780919304803409F43FC0BE
:1021D00050F4803221F18033A1F1813109F082C0C5
:1021E000F60110820AC0813509F458C0803809F41C
:1021F0006AC0803509F076C039C0D7018D919D91B4
:102200007D01009739F0DC01ED91FC910480F581AE
:10221000E02D0995EC14FD0481F782E161C00E9474
:102220009C0700918F0410919004209191043091AB
:102230009204DC01CB01801B910BA20BB30BB7FD09
:1022400051C061E088EE0E94DF0980E449C088EE59
:102250000E94CE0980FD46C088ED0E94CE09682FFD
:10226000686088ED0E94DF0980E53AC088EC0E9432
:10227000CE0986FF37C081E5809393040E949C07B6
:10228000DC01CB014496A11DB11D80938F04909376
:102290009004A0939104B093920424C00E949C07E0
:1022A000C0908F04D0909004E0909104F09092043C
:1022B000DC01CB018C199D09AE09BF09B7FD12C025
:1022C00080E8809393042C2F40E060E0C8010E94D6
:1022D0001E0F882321F0823D29F080EA01C080E9A9
:1022E00080939304CF911F910F91FF90EF90DF9017
:1022F000CF90BF90AF90089580E0089580E008955A
:1023000081E00895FC018285089581E0693009F03B
:1023100080E00895CF93DF93EC018A819B81DC01FB
:10232000ED91FC910480F581E02D6A8509958A85FF
:10233000813439F4EA81FB81EA58FF4F808184605F
:1023400080831A861B861C861D861E861F86188A19
:1023500080E0DF91CF9108958F929F92AF92BF92CC
:10236000CF92EF920F93A42EB12CB22A1F921F92FC
:102370001F921F921F921F92812C912CC12CE62E2E
:1023800001E023E240E0FC016285828193810E94AA
:102390005D0D0F900F900F900F900F900F900F9179
:1023A000EF90CF90BF90AF909F908F9008958F92B5
:1023B0009F92AF92BF92CF92EF920F93A62EB12C25
:1023C0001F921F923F932F935F934F934A01C12C0B
:1023D000E12C00E023EA40E0FC01628582819381E8
:1023E0000E945D0D0F900F900F900F900F900F9027
:1023F0000F91EF90CF90BF90AF909F908F900895E6
:102400008F929F92AF92BF92CF92EF920F93A42E92
:10241000B12CB22A1F921F921F921F921F921F92DD
:10242000812C912CC12CE62E03E023E240E0FC013C
:102430006285828193810E945D0D0F900F900F90B5
:102440000F900F900F900F91EF90CF90BF90AF90A3
:102450009F908F9008952F923F924F925F926F922C
:102460007F928F929F92AF92BF92CF92DF92EF9224
:10247000FF920F931F93CF93DF93CDB7DEB7E8970B
:102480000FB6F894DEBF0FBECDBFDC011A963C91AB
:10249000311107C1122F242E362E3C01FC01C280BF
:1024A000D380D601ED91FC910190F081E02D60E0A8
:1024B000C60109957C01009709F4F5C0FC01A080D4
:1024C000B180A114B10409F4F0C04301F4E08F0E0F
:1024D000911CDC0111969C928E9214961C93FE0125
:1024E00031962F018F0128E030E040E060E0D30119
:1024F00012968D919C9113970E943D0EF7011482C4
:102500008111D9C08D81893009F0D1C00981D601EE
:10251000ED91FC910280F381E02D222D41E0632DAD
:10252000C6010995F3018287882309F4C2C0988502
:102530009583282F40E060E0828193810E94B30E52
:10254000182F882389F0D701AD92BC92D601ED9166
:10255000FC910480F581E02DD3011A966C91C6019F
:102560000995F3011286ABC0202F013208F020E25A
:10257000D701AD92BC9221110BC0940142E0F3014E
:102580006285828193810E946D09811197C010C07C
:1025900030E0820140E0D3011A966C911A971296AE
:1025A0008D919C9113970E943D0E811187C0E5CFBC
:1025B0001F921F925F924F921F9288E08F9388E044
:1025C000882E912CA12CB12C99E2C92EE12C06E089
:1025D00020EA40E0F3016285828193810E945D0DD3
:1025E000182F0F900F900F900F900F900F90811158
:1025F00066C08B81D3011B968C931B97720100E000
:1026000028E030E040E01A966C911A9712968D916E
:102610009C9113970E94640E811150C02B813C81C4
:1026200040E0F3016285828193810E94640E8111F2
:1026300045C0298130E0CE0181967C0140E0D30184
:102640001A966C911A9712968D919C9113970E94ED
:10265000640E811133C02E8140E0F30162858281D6
:1026600093810E942110811129C001E0D3011B96A2
:102670008C91801740F020E0402F68E0C3010E9459
:1026800000120F5FF3CFD3011296ED91FC911397D7
:10269000EA58FF4F80818460808381E050968C935C
:1026A0000EC019ED0CC016ED0AC017ED08C011EDF3
:1026B00006C014ED04C0F701B182A082182F812F4B
:1026C000E8960FB6F894DEBF0FBECDBFDF91CF9175
:1026D0001F910F91FF90EF90DF90CF90BF90AF9040
:1026E0009F908F907F906F905F904F903F902F9032
:1026F0000895CF92DF92FF920F931F93CF93DF93B2
:1027000000D000D0CDB7DEB78C01F62E19821A8228
:102710001B821C8220E0462F61E10E94AC1120E068
:102720004F2D60E1C8010E94AC1120E04F2D64E004
:10273000C8010E94001283E0C82ED12C9E012F5F99
:102740003F4F44E050E06F2DC8010E94D71188230D
:10275000F1F020E04F2D64E1C8010E94AC1120E0AF
:102760004F2D60E1C8010E94AC1164E170E080E08F
:1027700090E00E949E070F900F900F900F90DF91B6
:10278000CF911F910F91FF90DF90CF900895898195
:102790009A81AB81BC819D7F83309140A041B1057E
:1027A000C1F264E670E080E090E00E949E0781E064
:1027B000C81AD10819F6CDCFFC0183E991E09183C5
:1027C0008083738362831286138614861586168629
:1027D0001786108A148288E085839CE3968391E0B3
:1027E0009783808784E0818761157105B1F0DB01F3
:1027F000AA5ABF4F80E090E02D913D91232B49F4E0
:102800008B96880F991FDB01A80FB91FED93FC93DE
:10281000089501968031910579F70895EF92FF921E
:102820000F931F93CF938C01C62F7A01FA018081F9
:102830009181A281B3818130F3E09F07F1E0AF077E
:10284000B105D1F060F48115E1E09E07AE07B10556
:1028500071F181309140A140B10571F064C08330C5
:1028600021E0920720E1A207B105E1F18330934016
:10287000A041B105B9F157C080919404811153C0B2
:1028800020E04C2F61E1C8010E94AC1120E04C2FE8
:1028900060E1C8010E94AC1120E04C2F64E0C80147
:1028A0000E94001281E08093940481EB3DC020E0FF
:1028B000462F61E1C8010E94AC1120E04C2F60E17D
:1028C000C8010E94AC1110929404F80162856770EF
:1028D000C770660F660F660F6C2B828193810E9412
:1028E0008A0921C020E04C2F64E1C8010E94AC118C
:1028F00020E04C2F60E1C8010E94AC1164E170E05F
:1029000080E090E00E949E07F8016285F701218136
:102910002695217067704C2FF801828193810E9467
:102920001E0F1092940480E0CF911F910F91FF90A1
:10293000EF900895CF92DF92EF920F931F93CF9372
:10294000DF93CDB7DEB72E970FB6F894DEBF0FBE7C
:10295000CDBF6C0181E090E09E878D87E12C8E01D8
:102960000F5F1F4F9E01235F3F4F41E0F6016285DD
:10297000828193810E944610811151C002E011E0D2
:1029800089818023D1F019861A861B861C869E01B8
:10299000275F3F4F44E050E0612FC6010E94D711EE
:1029A00081110BC0AE01475F5F4F612FC6010E94CE
:1029B0000E14813B99F1811132C0000F1F5F183056
:1029C000F9F611E0F6018385811740F119861A8620
:1029D0001B861C869E01275F3F4F44E050E0612F1D
:1029E000C6010E94D711811117C089859A85877009
:1029F00091708130914081F48B859C8581609C87AA
:102A00008B87AE01475F5F4F612FC6010E940E1496
:102A1000813B21F0811103C01F5FD4CF80E02E964F
:102A20000FB6F894DEBF0FBECDBFDF91CF911F91DF
:102A30000F91EF90DF90CF9008950F931F93CF9356
:102A4000DF93FC012089211102C080E020C0EC014D
:102A50000E949C070C851D852E853F85DC01CB01DE
:102A6000801B910BA20BB30BB7FDEFCFCE010E94E1
:102A70009A14182F0E949C07DC01CB018C599F4FA0
:102A8000AF4FBF4F8C879D87AE87BF87812FDF9168
:102A9000CF911F910F9108958091A10508950895F8
:102AA0000895CF93DF932091BE05243049F521E0AE
:102AB0002093E90021E8215059F03091E80035FDDC
:102AC00007C0EFE3F1E03197F1F700C00000F3CF6A
:102AD0002091E80025FF14C0EC0140E050E068E0E0
:102AE00070E00E9454198091E8008E778093E8008E
:102AF00088E0FE01A9E9B5E001900D928A95E1F721
:102B0000DF91CF910895CF93C0919704C1110BC06D
:102B10000E940108643C79408105910520F081E024
:102B200080939704C1E08C2FCF910895FF920F936B
:102B30001F93CF93DF93D82F0FB607FE83C08091EA
:102B4000BE05843081F08091040190E001962091CF
:102B5000060130E0822393232091050130E08217A3
:102B6000930709F0CDC00E948315811110C0809198
:102B7000040190E001962091060130E08223932326
:102B80002091050130E08217930709F0B9C00E9437
:102B9000F5078C01C091E900CF709091EC00892F6E
:102BA000817090FD80E8C82B82E08093E90085E089
:102BB000F82E8091EB0085FD42C08091EB0080FFF4
:102BC0003EC08091EE0087FF3AC080910501909150
:102BD0000401981709F457C09091E80095FF8EC042
:102BE000E0910201F0910301E80FF11D20818F5F58
:102BF000909106018923809305012093F100809133
:102C0000E80085FDE2CF8091E80080FFDECF809173
:102C1000E8008E778093E800F0920101D6CF809192
:102C2000040190E001962091060130E08223932375
:102C30002091050130E08217930709F44CC0CF7052
:102C4000C093E90040910401842F90E00196209107
:102C5000060130E0822393232091050130E08217A2
:102C6000930709F450C0E0910201F0910301E40FD1
:102C7000F11DD083809104018F5F9091060189231B
:102C80008093040140C08091E80085FF37C0D09355
:102C9000F10021E03091F3008091F20090E0932B5D
:102CA000892B91F08091E80080FF0EC08091E800B0
:102CB00085FF03C01092F100F9CF8091E8008E7774
:102CC0008093E800F0920101222309F4A8CFCF708D
:102CD000C093E90018C080910101882309F4AFCFA7
:102CE0000E94F5079C018017910711F4890161CFBB
:102CF00090910101915090930101F8CF20E0CACF4B
:102D000040910401B0CF80E0DF91CF911F910F91EE
:102D1000FF90089508958091BD05811104C00E941F
:102D2000BE1B0C941B1C08951092BD0508950895B8
:102D300042E061EC81E00E94CD1842E261EC82E069
:102D40000C94CD188091C005833009F453C030F441
:102D5000813071F0823009F4BAC008958A3009F4E4
:102D6000A6C08B3009F478C0893009F0C8C020C0F3
:102D70008091BF05813A09F0C2C08091E800877F49
:102D80008093E8008091C3059091C405892B21F4BC
:102D900068E089E995E003C060E080E090E070E0E1
:102DA0000E949F198091E8008B778093E800089536
:102DB0008091BF05813209F0A2C08091C305909136
:102DC000C405892B09F09BC08091E800877F809320
:102DD000E8008091E80082FD05C08091BE05811168
:102DE000F8CF8DC08091F1008093A1058091E8001B
:102DF0008B7781C08091BF05813A09F080C08091B6
:102E0000C3059091C405892BA1F48091E800877FC8
:102E10008093E8008091E80080FFFCCF8091120150
:102E20008093F1008091E8008E778093E8000E9403
:102E300002198091C3059091C405892B09F05FC0E8
:102E40008091E800877F8093E8008091E80080FF10
:102E5000FCCF809111014AC08091BF05813209F0F9
:102E60004EC08091C3059091C405892B69F480916F
:102E7000E800877F8093E8000E9402198091C105D5
:102E8000809312010E94C81E8091C3059091C405D1
:102E9000892BA9F58091E800877F8093E8000E9444
:102EA00002198091C105809311010C94C81E809174
:102EB000BF05813221F58091E800877F8093E8008B
:102EC0000E9402198091C2058093A2050895809105
:102ED000BF05813AA1F48091E800877F8093E800E4
:102EE0008091E80080FFFCCF8091A2058093F100E3
:102EF0008091E8008E778093E8000C940219089581
:102F00008091A105809398041092A1050E94D71D7D
:102F10000C94C81E0C9480170E94F5208091BC056B
:102F2000882329F00E941E2181110C94B71808955E
:102F30000E942621809198048093A10508950C9405
:102F400098170895CF9384B7877F84BF0FB6F894FE
:102F5000A895809160008861809360001092600065
:102F60000FBE90E080E80FB6F894809361009093D4
:102F700061000FBE86E995E10E948D2087E091E017
:102F80000E94501D8EE792E00E9427020E945B077C
:102F90000E94981D0E94BE1B0E941B1C78940E94D8
:102FA0009A1D8091BE05843019F00E94A117F9CFB7
:102FB0008CE692E00E9427020E946E068AE592E06B
:102FC0000E942702C2E08091BE05853019F40E945C
:102FD0008C17F9CF0E949E1D2091E4003091E500EE
:102FE00080919504909196042817390761F3809198
:102FF000E4009091E50090939604809395040E94DC
:103000008315882301F38091BE058430E1F6809119
:10301000E9008F702091EC00922F917020FD90E8D4
:10302000892BC093E9009091EB0090FF43C09091F1
:10303000EE0097FF3FC090910501209104012917F0
:1030400009F12091E80025FF1DC0E0910201F091F7
:103050000301E90FF11D30819F5F2091060192234A
:10306000909305013093F1009091E80095FDE3CF36
:103070009091E80090FFDFCF9091E8009E779093C9
:10308000E800D9CF9091F3002091F20030E0392B85
:10309000232B81F09091E80090FF0CC09091E80004
:1030A00095FF03C01092F100F9CF9091E8009E7750
:1030B0009093E8008F708093E90085CF292F332704
:1030C00023303105C9F060F42130310581F0223020
:1030D000310509F044C082E490E021ED32E043C0C4
:1030E00021323105E1F02232310549F138C082E167
:1030F00090E023E133E037C099278130910549F012
:1031000028F0029761F5E5E9F2E005C0EDECF2E0A8
:1031100002C0E3ECF2E0849190E09F0124C06115CD
:10312000710541F061307105D1F489E090E02CEF38
:1031300032E019C089E090E023EE32E014C061155E
:10314000710541F06130710551F482E290E025E2B1
:1031500033E009C080E490E027E433E004C080E07D
:1031600090E020E030E0FA0131832083089580E18F
:1031700089BD82E189BD09B400FEFDCF8091D800F0
:103180008F7D8093D8008091E00082608093E00082
:103190008091E00081FDFCCF0895982F973068F56D
:1031A0009093E900981739F07091EC002091ED00B0
:1031B0005091F00003C0242F762F50E021FD02C073
:1031C0009F5FECCF3091EB003E7F3093EB0030916E
:1031D000ED003D7F3093ED003091EB003160309396
:1031E000EB007093EC002093ED005093F0002091E1
:1031F000EE0027FDE5CF80E008958F708093E90011
:1032000081E008958091BF0587FF11C08091E8009B
:1032100082FD05C08091BE058111F8CF11C080915B
:10322000E8008B770BC08091BE05882349F0809120
:10323000E80080FFF8CF8091E8008E778093E80067
:1032400008952091E4003091E50095E64091EC006E
:10325000842F817040FF23C08091E80080FD1DC055
:103260008091BE05882399F0853099F08091EB001C
:1032700085FD11C04091E4005091E5002417350709
:1032800029F3915011F09A01E1CF84E0089582E092
:10329000089583E0089581E0089580E008954091C5
:1032A000E80042FFDDCF0895CF92DF92EF92FF92C8
:1032B0000F931F93CF93DF93EC018B017A010E9450
:1032C0002119811133C0E114F10439F0F701808133
:1032D0009181081B190BC80FD91FC12CD12C0115C6
:1032E000110519F18091E80085FD16C08091E80074
:1032F0008E778093E800E114F10449F0F7018081B2
:103300009181C80ED91ED182C08285E00FC00E9473
:103310002119882321F30AC089918093F10001507B
:103320001109FFEFCF1ADF0ADACF80E0DF91CF91EA
:103330001F910F91FF90EF90DF90CF900895209113
:10334000C5053091C6052617370748F06115710588
:1033500039F42091E8002E772093E80001C0B901EC
:10336000FC0120E06115710579F18091BE0588238B
:10337000F1F18530F1F18091E80083FD3CC080914E
:10338000E80082FD2EC08091E80080FFEBCF209105
:10339000F3008091F20090E0922B6115710551F0DD
:1033A0008830910538F421912093F1006150710922
:1033B0000196F3CF21E0089709F020E08091E80022
:1033C0008E778093E800CECF2111CFCF0AC08091B5
:1033D000BE05882361F0853061F08091E80083FDAF
:1033E0000AC08091E80082FFF2CF80E0089582E079
:1033F000089583E0089581E008952091C5053091F6
:10340000C6052617370748F06115710539F4209174
:10341000E8002E772093E80001C0B901FC0120E00C
:103420006115710591F18091BE05882309F440C0B2
:10343000853009F43FC08091E80083FD3DC0809154
:10344000E80082FD2FC08091E80080FFE9CF209145
:10345000F3008091F20090E0922B6115710559F014
:103460008830910540F424912093F1003196615009
:1034700071090196F2CF21E0089709F020E08091D0
:10348000E8008E778093E800CBCF2111CCCF0AC023
:103490008091BE05882361F0853061F08091E8005D
:1034A00083FD0AC08091E80082FFF2CF80E008959A
:1034B00082E0089583E0089581E008951F93CF93FB
:1034C000DF93CDB7DEB7AA970FB6F894DEBF0FBE75
:1034D000CDBFEFEBF5E08091F100819325E0E73C73
:1034E000F207C9F70E94A2168091E80083FF2EC15F
:1034F0008091BF059091C005492F50E04A30510599
:1035000008F024C1FA01EA5AFF4F0C94A423803832
:1035100021F0823809F01AC108C08091BB05909152
:10352000BC05992389F082600FC08091C3058F701C
:10353000873008F00BC18093E9008091EB0085FB98
:10354000882780F91092E9009091E800977F909386
:10355000E8008093F1001092F100D1C0282F2D7F58
:1035600009F0F4C0882319F0823061F0EFC0809137
:10357000C105813009F0EAC0933009F080E0809302
:10358000BC052EC08091C10581112AC08091C30560
:103590008F702FEF280F263008F0D8C08093E900F5
:1035A0002091EB0020FF1CC0933021F48091EB00B0
:1035B000806214C09091EB0090619093EB0021E049
:1035C00030E0A90102C0440F551F8A95E2F74093ED
:1035D000EA001092EA008091EB0088608093EB0093
:1035E0001092E9008091E800877F8093E8000E94B4
:1035F0000219ACC08111AAC01091C1051F7780913A
:10360000E3008078812B8093E3008091E800877F3E
:103610008093E8000E9402198091E80080FFFCCFAF
:103620008091E30080688093E300111102C082E082
:1036300001C083E08093BE0589C08058823008F0C5
:1036400085C08091C1059091C2058C3D53E09507DE
:1036500079F583E08A838AE289834FB7F894DE01A3
:10366000139620E03EE051E2E32FF0E05093570044
:10367000E49120FF03C0E295EF703F5FEF708E2F63
:1036800090E0EA3010F0C79601C0C0968D939D93EC
:103690002F5F243149F74FBF8091E800877F8093E7
:1036A000E8006AE270E0CE0101960E949F1916C000
:1036B0006091C3057091C405AE014F5F5F4F0E94DA
:1036C0005E18BC01892B09F441C09091E800977FF6
:1036D0009093E80089819A810E94FD198091E80009
:1036E0008B778093E80032C0803881F58091E800C4
:1036F000877F8093E8008091BA058093F1008091E4
:10370000E8008E7772CF811121C08091C105909120
:10371000C20599270297D4F48091E800877F8093AF
:10372000E8008091C1058093BA050E94021980913A
:10373000BA05811106C08091E30087FD02C081E0D7
:1037400001C084E08093BE050E9498168091E80035
:1037500083FF0AC08091E800877F8093E800809112
:10376000EB0080628093EB00AA960FB6F894DEBF60
:103770000FBECDBFDF91CF911F9108950E942C1CE9
:103780000E94341CE0EEF0E0808181608083E8EDEF
:10379000F0E080818F77808319BCA7EDB0E08C9139
:1037A0008E7F8C9380818F7E80831092BD050895DB
:1037B0000F931F93CF93DF930E942C1C0E94341C05
:1037C000C8EDD0E088818F7788838881806888837E
:1037D00088818F7D888319BC1092BE051092BA052E
:1037E0001092BC051092BB0500EE10E0F80180813C
:1037F0008B7F808388818160888342E060E080E005
:103800000E94CD18E1EEF0E080818E7F8083E2EEB1
:10381000F0E0808181608083808188608083F8010E
:1038200080818E7F8083888180618883DF91CF91C2
:103830001F910F910895E8EDF0E080818F7E8083E5
:10384000E7EDF0E080818160808384E082BF81E0E9
:103850008093BD050C94D81BE8EDF0E080818E7F4D
:1038600080831092E20008951092DA001092E10035
:1038700008951F920F920FB60F9211242F933F932A
:103880004F935F936F937F938F939F93AF93BF9368
:10389000EF93FF938091E10082FF0BC08091E200E3
:1038A00082FF07C08091E1008B7F8093E1000E943E
:1038B0004F1D8091DA0080FF1FC08091D80080FFEB
:1038C0001BC08091DA008E7F8093DA008091D9004E
:1038D00080FF0DC080E189BD82E189BD09B400FE91
:1038E000FDCF81E08093BE050E948B1605C019BCF8
:1038F0001092BE050E9494168091E10080FF19C0CD
:103900008091E20080FF15C08091E2008E7F80935D
:10391000E2008091E20080618093E2008091D80013
:1039200080628093D80019BC85E08093BE050E9418
:103930008A178091E10084FF30C08091E20084FF0B
:103940002CC080E189BD82E189BD09B400FEFDCFB4
:103950008091D8008F7D8093D8008091E1008F7E88
:103960008093E1008091E2008F7E8093E20080915D
:10397000E20081608093E2008091BA05882311F013
:1039800084E007C08091E30087FD02C081E001C0B0
:1039900083E08093BE050E949F178091E10083FF22
:1039A00029C08091E20083FF25C08091E100877FDC
:1039B0008093E10082E08093BE051092BA05809169
:1039C000E1008E7F8093E1008091E2008E7F809302
:1039D000E2008091E20080618093E20042E060E0DA
:1039E00080E00E94CD188091F00088608093F00004
:1039F0000E949716FF91EF91BF91AF919F918F9188
:103A00007F916F915F914F913F912F910F900FBEDA
:103A10000F901F9018951F920F920FB60F921124BE
:103A20002F933F934F935F936F937F938F939F93C6
:103A3000AF93BF93CF93DF93EF93FF93C091E900D0
:103A4000CF708091EC00D82FD17080FDD0E810921B
:103A5000E9008091F000877F8093F00078940E94C5
:103A60005E1A1092E9008091F00088608093F00067
:103A7000CD2BCF70C093E900FF91EF91DF91CF91F3
:103A8000BF91AF919F918F917F916F915F914F9176
:103A90003F912F910F900FBE0F901F901895089592
:103AA0009093A8058093A7050895E091A705F0914C
:103AB000A805309721F00190F081E02D099480E075
:103AC0000895E091A705F091A805309721F00280B4
:103AD000F381E02D099408952091A5053091A60564
:103AE0002817390771F09093A6058093A505E091FA
:103AF000A705F091A805309721F00680F781E02D09
:103B0000099408952091A3053091A4052817390739
:103B100071F09093A4058093A305E091A705F0911F
:103B2000A805309721F00084F185E02D09940895CF
:103B30000C94D81D0E94EC070C946D06CF93DF9374
:103B400000D000D01F92CDB7DEB70E9475068FEF70
:103B500089838A831B820E94F5078160782F9D8369
:103B60008C8349815A816B818D810E94781F0E94CC
:103B700077060E94551D9091A905891769F00E944A
:103B8000551D8093A9050F900F900F900F900F90E7
:103B9000DF91CF910C94F1200F900F900F900F9028
:103BA0000F90DF91CF91089508950C94D41D08953E
:103BB000089508950895882309F4BBC09CEF980FD9
:103BC000913A18F40E94FB1F0DC090E2980F9830B4
:103BD00058F4877091E001C0990F8A95EAF7892F10
:103BE0000E9436200C9467209BE5980F933070F468
:103BF000853A29F0863A31F083E890E005C081E803
:103C000090E002C082E890E00C946C1D98E5980F5B
:103C1000973108F08EC0883A09F445C0893A09F412
:103C200045C08A3A09F445C08B3A09F445C08C3A3C
:103C300009F445C08D3A09F445C08E3A09F445C0EF
:103C40008F3A09F445C0813B09F445C0803B09F433
:103C500045C0823B09F445C0833B09F445C0843B21
:103C600009F445C0853B09F445C0863B09F445C0CD
:103C7000873B09F445C0883B09F445C0893B09F4FA
:103C800045C08A3B09F445C08B3B09F445C08C3BD9
:103C900009F445C08D3B09F445C08E3B09F445C08D
:103CA00080E090E044C082EE90E041C089EE90E078
:103CB0003EC08AEE90E03BC085EB90E038C086EBDA
:103CC00090E035C083EB90E032C084EB90E02FC0F1
:103CD00087EB90E02CC08CEC90E029C08DEC90E05C
:103CE00026C083E891E023C08AE891E020C082E901
:103CF00091E01DC084E991E01AC081E292E017C012
:103D000083E292E014C084E292E011C085E292E086
:103D10000EC086E292E00BC087E292E008C08AE221
:103D200092E005C08FE690E002C080E790E00C943E
:103D3000821D0895882329F19CEF980F913A18F479
:103D40000E9418200DC090E2980F983058F48770A8
:103D500091E001C0990F8A95EAF7892F0E943C20D3
:103D60000C9467209BE5980F933020F480E090E05E
:103D70000C946C1D885A873120F480E090E00C94FC
:103D8000821D08950E9453200E9428200C946720D1
:103D90000E9443200C94C21EEF92FF920F931F9338
:103DA000CF93DF9300D000D01F92CDB7DEB78C0148
:103DB0000E94F320811190C085E0F801DE01119688
:103DC00001900D928A95E1F7F8014081518123819C
:103DD00034812115310531F05F3F31F481E04F3FEF
:103DE00019F403C081E001C080E080FD75C0F801D6
:103DF000E28049835A83EB82722F3D832C836E2DA0
:103E00008D810E94B51FF82E492F4F70892F829502
:103E10008F708E30B1F108F050C0823008F05CC075
:103E2000907F142F11F01295107FEE20A9F011232E
:103E300029F0812F0E9446200E9467208F2D0F902D
:103E40000F900F900F900F90DF91CF911F910F91D6
:103E5000FF90EF900C94DB1D8F2D0E949A1E112372
:103E6000D9F1812F0E944C200F900F900F900F904E
:103E70000F90DF91CF911F910F91FF90EF900C94D5
:103E80006720F11029C0EE2039F10E94C81EFFEF13
:103E900020E782E0F15020408040E1F700C00000C0
:103EA0000F900F900F900F900F90DF91CF911F9177
:103EB0000F91FF90EF900C9453216F2DC8010F903C
:103EC0000F900F900F900F90DF91CF911F910F9156
:103ED000FF90EF900C9472210F900F900F900F9025
:103EE0000F90DF91CF911F910F91FF90EF90089568
:103EF000CF93DF93CDB7DEB72A970FB6F894DEBF26
:103F00000FBECDBF942F4E83252F5F83688779879F
:103F10008A8749855A85452B31F02F3F31F481E05E
:103F20009F3F19F403C081E001C080E080FD07C01D
:103F30004E815F81688579858A850E94E22085E0CF
:103F4000FE013696DE01119601900D928A95E1F7F9
:103F5000CE0101960E94CC1E2A960FB6F894DEBFC1
:103F60000FBECDBFDF91CF9108950F931F93CF93D5
:103F7000DF9300D000D01F92CDB7DEB7042F498366
:103F80005A836B837C838D832C813D81232B31F07D
:103F90005F3F31F481E04F3F19F403C081E001C07D
:103FA00080E080FF03C080E090E01BC08B8110E0C8
:103FB000882379F06091AA057091AB058091AC05DA
:103FC0009091AD050E949220F801E655FA4F80834A
:103FD00004C0F801E655FA4F808169817A810E9418
:103FE00082210F900F900F900F900F90DF91CF9143
:103FF0001F910F9108952091130130911401F9013F
:1040000032969FEF40E05191851789F09F3F19F458
:10401000511101C0942F4F5F4630A9F79F3F39F0EF
:10402000F901E90FF11D97FDFA958283089508952E
:10403000E0911301F09114019F012A5F3F4F92819B
:10404000891301C012823196E217F307C1F7089570
:1040500081E090E0E0911301F0911401E80FF91F65
:104060001082019688309105A9F708959091B805BE
:10407000892B8093B805089580959091B805892380
:104080008093B80508951092B80508959091B705EA
:10409000892B8093B705089580959091B705892362
:1040A0008093B70508951092B70508958091130184
:1040B00090911401FC0131969C01285F3F4F80E0F4
:1040C000919191118F5FE217F307D1F70895E09175
:1040D0001301F09114018091B8058083E0911301E0
:1040E000F091140190818091B705892B8083809194
:1040F000AE05882361F0E0911301F09114019081E5
:10410000892B80830E94562081111092AE058091E8
:104110001301909114010C94611D9093A701809359
:10412000A6010895CF92DF92EF92FF926C01EE24E8
:10413000FF24C114D104E104F10421F0C701B60148
:1041400020E101C020E0C72ED82EE92EFF24C114A3
:10415000D104E104F10419F0285FC701B6016B0135
:104160007C0154E0F694E794D794C7945A95D1F71C
:10417000C114D104E104F10419F02C5FC701B601A8
:104180006B017C0142E0F694E794D794C7944A957A
:10419000D1F7C114D104E104F10419F02E5FC70175
:1041A000B601DC01CB01B695A79597958795892B2C
:1041B0008A2B8B2B09F02F5F822FFF90EF90DF90DF
:1041C000CF900895CF93DF9300D000D01F92CDB74A
:1041D000DEB70F900F900F900F900F90DF91CF915F
:1041E00008950C94D51D80E008958091BE0584301B
:1041F00021F11092B90520E488E190E00FB6F8941F
:10420000A895809360000FBE2093600083B7817FE4
:10421000846083BF83B7816083BF7894889583B7B8
:104220008E7F83BF0FB6F894A89580916000886157
:1042300080936000109260000FBE08950E94D91D07
:104240000E9475060E94DA1D80E008950E94D71D25
:104250000C94C81E1F920F920FB60F9211248F93C9
:104260009F93AF93BF938091B905811113C0809143
:104270008B0490918C04A0918D04B0918E04419692
:10428000A11DB11D80938B0490938C04A0938D0489
:10429000B0938E04BF91AF919F918F910F900FBEFD
:1042A0000F901F9018950E94BE1BF89487E797E720
:1042B000909301088093000887E090EBDC018093E5
:1042C000C7059093C805A093C905B093CA059CE0A3
:1042D00088E10FB6F894A895809360000FBE909384
:1042E0006000FFCF0895E62FF0E0EB5AFD4F849178
:1042F0000895E82FF0E0EE0FFF1FED52FF4F85917C
:10430000949108950E94732190E4980F903218F4CC
:104310000E94792108958F3B50F4883A48F5853AF8
:10432000D0F48430A8F4813009F4B2C0AEC0883E25
:1043300040F4803E68F48F3B09F0A7C020E030EEE7
:10434000A9C0803F08F4A1C0282F30E03065A2C08A
:10435000282F30E09FC0853A29F0863A31F023E8D3
:1043600030E498C021E830E495C022E830E492C0FF
:10437000883A09F445C0893A09F445C08A3A09F4F3
:1043800045C08B3A09F445C08C3A09F445C08D3AD2
:1043900009F445C08E3A09F445C08F3A09F445C086
:1043A000813B09F445C0803B09F445C0823B09F4D8
:1043B00045C0833B09F445C0843B09F445C0853BB7
:1043C00009F445C0863B09F445C0873B09F445C064
:1043D000883B09F445C0893B09F445C08A3B09F490
:1043E00045C08B3B09F445C08C3B09F445C08D3B6F
:1043F00009F445C08E3B09F445C020E034E44AC0CE
:1044000022EE34E447C029EE34E444C02AEE34E41A
:1044100041C025EB34E43EC026EB34E43BC023EB43
:1044200034E438C024EB34E435C027EB34E432C044
:104430002CEC34E42FC02DEC34E42CC023E835E41C
:1044400029C02AE835E426C022E935E423C024E95E
:1044500035E420C021E236E41DC023E236E41AC070
:1044600024E236E417C025E236E414C026E236E43E
:1044700011C027E236E40EC02AE236E40BC02FE674
:1044800034E408C020E734E405C020E030E002C096
:1044900021E030E0C90108950E94BD2208F481E0C6
:1044A00008950E94112388F09F5798F0B92F9927FB
:1044B000B751B0F0E1F0660F771F881F991F1AF00F
:1044C000BA95C9F714C0B13091F00E942B23B1E026
:1044D00008950C942B23672F782F8827B85F39F025
:1044E000B93FCCF3869577956795B395D9F73EF4A8
:1044F00090958095709561957F4F8F4F9F4F089550
:10450000E89409C097FB3EF490958095709561956D
:104510007F4F8F4F9F4F9923A9F0F92F96E9BB2723
:104520009395F695879577956795B795F111F8CF9F
:10453000FAF4BB0F11F460FF1BC06F5F7F4F8F4F0A
:104540009F4F16C0882311F096E911C0772321F000
:104550009EE8872F762F05C0662371F096E8862F98
:1045600070E060E02AF09A95660F771F881FDAF7EF
:10457000880F9695879597F90895990F0008550F1C
:10458000AA0BE0E8FEEF16161706E807F907C0F0D9
:1045900012161306E407F50798F0621B730B840BE1
:1045A000950B39F40A2661F0232B242B252B21F4BB
:1045B00008950A2609F4A140A6958FEF811D811D5B
:1045C000089597F99F6780E870E060E008959FEF95
:1045D00080EC089500240A9416161706180609069A
:1045E000089500240A941216130614060506089569
:1045F000092E0394000C11F4882352F0BB0F40F4F1
:10460000BF2B11F460FF04C06F5F7F4F8F4F9F4F30
:10461000089557FD9058440F551F59F05F3F71F0B2
:104620004795880F97FB991F61F09F3F79F0879519
:104630000895121613061406551FF2CF4695F1DFA2
:1046400008C0161617061806991FF1CF8695710532
:10465000610508940895E894BB2766277727CB0166
:1046600097F908950E94BD2208F48FEF08950E94E3
:104670004A230C94F8220E94EA2238F00E94F12288
:1046800020F0952311F00C94E1220C94E7221124E0
:104690000C942C230E94092370F3959FC1F3950F6E
:1046A00050E0551F629FF001729FBB27F00DB11DB6
:1046B000639FAA27F00DB11DAA1F649F6627B00D46
:1046C000A11D661F829F2227B00DA11D621F739F2F
:1046D000B00DA11D621F839FA00D611D221F749F3D
:1046E0003327A00D611D231F849F600D211D822F84
:1046F000762F6A2F11249F5750409AF0F1F08823AB
:104700004AF0EE0FFF1FBB1F661F771F881F9150D7
:104710005040A9F79E3F510580F00C94E1220C9483
:104720002C235F3FE4F3983ED4F386957795679505
:10473000B795F795E7959F5FC1F7FE2B880F911D01
:104740009695879597F90895EE0FFF1F0590F491C0
:08475000E02D0994F894FFCF5D
:10475800010599040000FF4C1551154F158A165094
:10476800150101AF052F2F20556E6B6E6F776E20E8
:10477800484944204465736320547970653A002F92
:104788002F20556E6B6E6F776E20446573632054CF
:104798007970653A00206C656E002F2F2069645689
:1047A800656E646F72002F2F20696450726F647594
:1047B8006374002F2F206C616E676964000000002D
:1047C80000D602000000007A078007760779077094
:1047D8000773077307000000009B084208FB0800E6
:1047E8000000002B127C118A111D15821179137E8D
:0647F80011851180110083
:00000001FF
